:1000000003C003C003C003C003C003C003C003C0D8
:1000800033C0000049C0000047C0000045C0000068
:1000900043C0000041C000003FC000003DC0000060
:1000A0003BC0000039C0000037C0000035C0000070
:1000B00033C0000031C000002FC000002DC0000080
:1000C0002BC0000029C0000027C0000025C0000090
:1000D00023C0000021C000001FC000001DC00000A0
:1000E0001BC0000019C0000000000000000000005C
:1000F0000000000000000000000000000000000000
:10010000000000000000000011241FBECFEFD4E06B
:10011000DEBFCDBFFDD315C4B3CF009709F408955A
:10012000E0EAFFE03197F1F70197F7CF80789B0184
:1001300020583F4FDB01FC01E61BF70BEA0FFB1FCA
:10014000459154914D935D93A217B307A1F708957C
:10015000FC01E07893E090935700E89507B600FC27
:10016000FDCF0895CF93DF939B0120583F4FDB01D4
:10017000FC01E61BF70BEA0FFB1FCD91DD9141E07F
:100180000E0140935700E8951124A217B30781F799
:1001900025E0FC0120935700E89507B600FCFDCF51
:1001A000DF91CF910895CF93DF93CDB7DEB7C058DD
:1001B000D1090FB6F894DEBF0FBECDBFBE016F5F91
:1001C0007F4F90E080E0B2DFFE013196CE018F5785
:1001D0009F4F2FEF3FEF21933193E817F907C9F7AE
:1001E00090E080E0B5DFBE016F5F7F4F90E080E080
:1001F000B9DFC058DF4F0FB6F894DEBF0FBECDBFDA
:10020000DF91CF910895EF92FF920F931F93CF93B9
:10021000DF93CDB7DEB7C058D1090FB6F894DEBF73
:100220000FBECDBF10E000E045E00A3D140774F0BA
:10023000C058DF4F0FB6F894DEBF0FBECDBFDF91C1
:10024000CF911F910F91FF90EF90089530E020E043
:10025000F801EA5CFC4FE20FF31FC9018E7F49E011
:10026000E031F407ECF44591549161E070E06C0FDB
:100270007D1F860F971FFC01518340832E5F3F4FE8
:100280002038310529F77801F6ECFF1AC70160DF45
:10029000BE016F5F7F4FC70165DF00581F4FC4CF9E
:1002A00041E050E04C0F5D1F840F951F4FEF5FEF53
:1002B000E2CF0F931F93CF93DF93CDB7DEB7C05834
:1002C000D1090FB6F894DEBF0FBECDBFFE01319647
:1002D000CE018F579F4F8F012FEF3CED219331932C
:1002E000E817F907C9F790E080E032DFB80190E045
:1002F00080E038DFC058DF4F0FB6F894DEBF0FBE86
:10030000CDBFDF91CF911F910F910895CF9384B10D
:10031000836084B92998CAEF81E090E0FEDE299AD3
:1003200081E090E0FADE2998C150B1F7CF910895AD
:10033000F0E0E0E0099417C0000039FC8005940B60
:1003400000000902120001010080320904000000CF
:100350000000000012011001FF000008D016530732
:1003600006020000000111241FBECFEFD4E0CDBF74
:10037000DEBF11E0A0E0B1E0ECE8FFE302C00590D1
:100380000D92AE34B107D9F721E0AEE4B1E001C07F
:100390001D92AA37B207E1F736C1DC0180E090E098
:1003A00041E050EA609530E009C02D918227979591
:1003B000879510F084279527305EC8F36F5FA8F308
:1003C0008D939D930895CF93DF93CC27C395319B55
:1003D000E9F7319B0BC0319B09C0319B07C0319BB2
:1003E00005C0319B03C0319B01C089C00F92C091F1
:1003F0005C01DD27CC59DE4F0F9065E5319B03C0D2
:100400000F920F90E6CF0F930F910F9320E040E1F2
:100410000F9106B1067001FB27F93F9350E03BE0D6
:1004200039C0167040642F77012F5F5F1EC040688F
:1004300016B116702F7752501FC0406406B12F7747
:100440000670D1F15F5F00C023C0406216B12F7704
:10045000167091F15F5F00C025C0067010275150E3
:1004600012F45D5F0000115027952C3F16B1C8F6BD
:1004700016700127015027952C3FC8F64227499353
:1004800006B1067010274F73115027952C3FA8F620
:100490004695469516B1167079F0012701502795BB
:1004A0002C3F98F66B5A60F3315006B1B0F600C09D
:1004B00012E01BBB00271DC03B503195C31BD04031
:1004C00012E01BBB0881033CE9F00B34D9F020910A
:1004D0005A011981110F1213EDCF093611F10D32A6
:1004E00011F0013E39F7CAE01BB311FD02C0CA95F5
:1004F000D9F7009362013F91CBB3C1FD67CFDF9184
:10050000CF910895209162012223A9F310916001F7
:10051000112309F534300AF13093600120935B0117
:100520001CC0009160010130B4F40AE530915D0116
:1005300034FD14C000935D01CFE4D1E013C0052762
:1005400010E000C0000008B91AC0052710E0221F03
:100550001DC010E021C04AE502C032ED432FC4E1C6
:10056000D0E032E017B11660419A08B117B956E0F1
:1005700020E865E320FF052708B9279517951C3F5C
:10058000F0F66695B8F7B1F720FF052708B927956B
:1005900017951C3FD0F62795179517FF05270000E4
:1005A0001C3F08B9B0F629913A9519F7097F1091C7
:1005B0006101110FC651D04008B911F010935A01D2
:1005C00012E01BBB026017B1197F402F497F54E036
:1005D0005A95F1F708B917B948B98DCFF20130979C
:1005E00079F0E230F10511F480E09DE121E00C01A9
:1005F00020935700E8951124CF0102962C0108950D
:100600008CE094E9F3CFA89514BE809160008861D6
:100610008093600010926000399A88EB9BE0E0E9DB
:10062000F1E03197F1F70197D1F739988AE5809396
:100630005D018FEF80934E0180916C008460809308
:100640006C0080916800826080936800519A712CE0
:10065000312C512C412CC5EDD4E184E696B1967035
:1006600009F084E6815021F41092610110925A0140
:10067000D99BA6C0A8DE82E08BBBA89522E03212EF
:100680000FC0E0E0FAE3E058F10983E080935700FF
:10069000E89507B600FCFDCF3097A9F7512C412C07
:1006A000832D803409F090C0F2013297E1158AE37E
:1006B000F80738F485E080935700E89507B600FC0A
:1006C000FDCF312C80916001835087FD2BC090912C
:1006D0005B019D3229F5883019F583EC80934F0139
:1006E0008AE580935D018091650180769091660135
:1006F000882309F4A7C0712C91117EC084E09AE38D
:1007000090935F0180935E0188E090916C0191115C
:1007100005C090916B01981708F4892F80934E01C2
:100720001092600180915D0184FF30C080914E0184
:100730008F3F61F1C82F893008F0C8E0982F9C1BCB
:1007400090934E0190914F0128E8922790934F018A
:10075000882381F0E0915E01F0915F01A0E5B1E0B6
:100760008C2F94919D9331968150D9F7F0935F012E
:10077000E0935E016C2F80E591E00FDECC5FCC3022
:1007800019F08FEF80934E01C0935D01C301019674
:100790003C01803921E0920729F4EDEFF9E3E4917F
:1007A000EF3FC1F48C7409F488C05998D99B53CF9A
:1007B0008CE1319B8CE18150E1F782E08BBB4BCF28
:1007C000219709F04BCF59CF843009F07ACFCD2B48
:1007D00009F078CF5198599880E091E08752914084
:1007E00009F06DC017B81092680010926C0081E19A
:1007F00080935700E8959DCD913079F441145104D0
:1008000011F480E082CF809169018078482E509069
:100810006A0181E187BFE895F4CF933081F480913C
:10082000670190916801DADE8091690190916A0117
:10083000D5DE842D8F7729F790E4392E66CF9F730C
:10084000392EDFCF209167011092580191110AC013
:100850001092590128E531E082E030935F01209346
:100860005E0153CF953029F42093610128E531E0F2
:10087000F4CF963091F480916801813041F48EE19B
:100880009AE390935F0180935E0182E13ECF8230D4
:1008900009F0B7CF8CE09AE3F4CF983051F099305B
:1008A00019F420936301E2CF81E09A30F9F280E0FD
:1008B000DDCF23E631E081E0D0CF599A77CF399868
:1008C00092CF282A28766F6C6174696C65207569EF
:1008D0006E74385F74202A29282830783037292010
:1008E0002B2030783230292900282A28766F6C6135
:1008F00074696C652075696E74385F74202A2928C4
:10090000283078304129202B2030783230292900B6
:1009100085B115B884B18FEF84B98AEF90E0FDDB23
:1009200084B114B88AEF90E0F8DBF8943CDC6BDC1F
:10093000C0DCECDC8DEF99E30BDCFADC90E080E0CE
:060940000895F894FFCFBA
:040000030000008079
:00000001FF
